:020000020000FC
:1000000009C0189543573732207665722E302E314D
:10001000342020207BD054D040B3417069F040B3ED
:10002000427049F14DD045D06623B1F36A95A1F7EE
:10003000C1983FD0C29AF0CFC19AC2983AD0C09826
:10004000C398882705E01FE034D0819B82601A9511
:10005000D9F70A95C1F7C09AC39A05E01DE029D0E7
:10006000819B82601A95D9F70A95C1F7482F427093
:1000700011F46FEFD1CFC19AC298C098C398882766
:100080000FE01FE016D0809B81601A95D9F70A9582
:10009000C1F7C09AC39A05E01DE00BD0809B816038
:1000A0001A95D9F70A95C1F7482F417029F66FEFD5
:1000B000B3CF2F2D30E83A95F1F72A95D9F7089567
:1000C00040B34695469546954F704E15F1F0E42E97
:1000D0005FE04030C9F05EE04130B1F05DE04230B9
:1000E00099F05CE0433081F05BE0443069F05AE025
:1000F000453051F059E0463039F058E0473021F0B2
:1001000057E0483009F056E0F52E08954FEF47BB11
:1001100044E741BB4DE048BB4FE742BB8827662719
:02012000089540
:00000001FF
